:100000000C94280018950000189500001895000021
:10001000189500001895000018950000189500002C
:10002000189500000C949B0D189500001895000081
:10003000189500001895000018950000189500000C
:1000400018950000189500001895000018950000FC
:100050008FE181BD87E181BD8FE58DBFC4E0E8E719
:100060004E2E88E08EBFD8E0F7E05F2EEEEFF7E08F
:10007000A0E6B0E088278D933197E9F783E389B94B
:1000800088E18AB9662481E48ABB81E38BBB8FEB6C
:1000900087BB8FEB88BB88E084BB83E085BB80E0B7
:1000A00081BB8BE382BB80E08FBD81E08EBD8FE1A1
:1000B00081BD87E181BD86E086B980E487B9C398B8
:1000C000C29AD89ADE9AC498C798C598F894A89509
:1000D0007091D100777F7093D1007091D1007B7FB8
:1000E0007093D1000027A1EDB0E08C9183FB0EF45A
:1000F00001E041E0041781E009F080E08F930027E0
:10010000A1EDB0E08C9182FB0EF401E041E0041718
:1001100081E009F080E09F91892B882311F40C94F1
:100120009400DC9881E58ABB0E940A0F7091D1008F
:1001300070627093D100EFEFF1E0A2ECB0E091E0DB
:100140000E94C22F0091C200003081E009F080E0DF
:100150008F930091C2000E3F80E010F009F081E023
:100160009F91892B882311F40C94B9008EEB809316
:10017000C2000091C2004AE0040F01BF89E190E093
:100180000E94B42EEAEDFFE50E94FB2D0027A1EDB1
:10019000B0E08C9183FB0EF401E041E0041711F014
:1001A0000C94DA00E6EFFFE50E94FB2D0E94072E7B
:1001B0000C94ED00E8EFFFE50E94FB2DA1EDB0E00F
:1001C0008C9182FBA8E6B7E00E94D92E8D938827F8
:1001D0008C930E94F32D0E94072EEAE0F0E0BB27EB
:1001E000A0E10E94BF2F073411F40C942D01EBE025
:1001F000F0E0A0E1BB278FE08C937BE70E94AE2F5D
:10020000ECE0F0E001E010E0A0E1BB277BE70E941A
:10021000B02FEAE0F0E0A0E1BB2787E48C937BE716
:100220000E94AE2FEEE0F0E0A0E1BB2780E08C93CF
:100230007BE70E94AE2FE0E1F0E000E010E0A0E1FB
:10024000BB277BE70E94B02FEFE0F0E0A0E1BB27E7
:1002500080E08C937BE70E94AE2FEBE0F0E0ABEB0D
:10026000B0E00E94BF2F0091BB00043618F011F0DF
:100270000C943C010C943F0184E68093BB0080E722
:1002800097E9ACEBB0E08D939C93ECE0F0E0A6EB4B
:10029000B0E00E94C12FEEE0F0E0A3ECB0E00E94DD
:1002A000BF2FEFE0F0E0A4ECB0E00E94BF2F0E946F
:1002B0000E0FE0E1F0E0A3E6B0E00E94C12FA3E65C
:1002C000B0E00E94622DE0E1F0E0A3E6B0E07BE761
:1002D0000E94B02FA6EBB0E00D911C91003050E0D1
:1002E000150711F00C947A0181E090E0A6EBB0E0E4
:1002F0008D939C93EAEFFFE50E94FB2DA8E6B7E003
:10030000EBEBF0E00E94472F0E94F32DE2E0F0E6D5
:100310000E94FB2DA8E6B7E0E6EBF0E00E94382F44
:100320000E94F32DE2E0F0E60E94FB2DA8E6B7E084
:10033000E3ECF0E00E94472F0E94F32DE2E0F0E6AC
:100340000E94FB2DA8E6B7E0E4ECF0E00E94472F06
:100350000E94F32DE2E0F0E60E94FB2DA8E6B7E054
:10036000E3E6F0E00E94382F0E94F32D0E94072E52
:1003700080E08093D00070916A00777F70936A006C
:1003800080E08093C60086E08093BE008DE080937D
:10039000BF00E9E6F0E0FA93EA930E94601E22961D
:1003A00084E190E00E94B42EDE980E94A02EC49AB0
:1003B000E4E0F0E60E94FB2D0E94072E88EC90E01E
:1003C0000E94B42EA89581B5886181BD877F81BDCB
:1003D000E0E6F0E0FA93EA930E9470222296A89554
:1003E00000916000003011F40C9402020E948421FC
:1003F000EEE0F0E60E94FB2D0E94072E0E94D10E37
:100400000C9407027091D1007F7B7093D100E8E1DA
:10041000F0E60E94FB2D0E94AD2184E690E00E9450
:10042000B42E00916900003018F011F00C941A02FB
:100430000C942102E9E6F0E0FA93EA930E94891F06
:1004400022960027A1EDB0E08C9186FB0EF401E02E
:1004500040E0041711F00C942F020E949D158FEFBD
:100460000E940A2E82E390E00E94B42E7894A89510
:1004700081B5886081BDA2EBB0E04D915C91A6EBA7
:10048000B0E00D911C910417150718F011F00C94B1
:100490004B020C94510281E090E0A6EBB0E08D930A
:1004A0009C930027AAE6B0E08C9184FB0EF401E057
:1004B00041E0041781E009F080E08F930027A1ED6F
:1004C000B0E08C9186FB0EF401E040E0041781E07F
:1004D00009F080E09F918923882311F40C94830212
:1004E000E6EBF0E0FA93EA935A924A9280E0A42D68
:1004F000B52D8C9381E00E944F2D0E944B132496C2
:1005000081E00E944B2DA895E1E0F0E00E940E2EC4
:10051000A895E1E0F0E00E940E2EA895E1E0F0E061
:100520000E940E2EA89580E08093B80080E0809312
:10053000690070916A007F7770936A000027A1EDCF
:10054000B0E08C9186FB0EF401E041E0041711F05D
:100550000C94AC020E940A0FA895ABE6B0E0882785
:100560008C930027A1EDB0E08C9183FB0EF401E0A9
:1005700041E0041711F00C94C4020E94EB2DABE68D
:10058000B0E08D9388278C93ABE6B0E08C918030FF
:1005900011F00C9497050091D000003081E009F033
:1005A00080E08F930027AAE6B0E08C9181FB0EF4E7
:1005B00001E040E0041781E009F080E09F91892B81
:1005C000882311F40C946704E0E6F0E0FA93EA93D0
:1005D0000E94B81E229600916000003018F011F0C1
:1005E0000C94F4020C94670470916A007068709324
:1005F0006A000091D200003011F00C945003409139
:10060000C60000916000041718F011F00C940A0362
:100610000C945003809160008093C6000027AAE6E6
:10062000B0E08C9184FB0EF401E040E0041711F07F
:100630000C942A03A0E6B0E08C91A6EBB0E08D9379
:1006400088278C93ABE6B0E0E2E2F0E60E94DA2D78
:100650000C9450030027A1EDB0E08C9187FB0EF4C1
:1006600001E041E0041711F00C944A03A0E6B0E069
:100670000D91112741E050E0040F151FA6EBB0E0EB
:100680000D931C93ABE6B0E0E2E2F0E60E94DA2DB7
:100690000C945003ABE6B0E0E4E2F0E60E94DA2D01
:1006A0000091D200013011F00C94E403009160003D
:1006B000013011F00C946203ABE6B0E0E4E2F0E646
:1006C0000E94DA2D00916000023011F00C946E034C
:1006D000ABE6B0E0E6E2F0E60E94DA2D80E080933F
:1006E000620000916000033081E009F080E08F93A8
:1006F0000091BB00043681E008F080E09F918923DF
:10070000882311F40C948C03ABEBB0E08C918E5FDA
:100710008C9381E08093620000916000043081E05E
:1007200009F080E08F930091BB00023080E010F070
:1007300009F081E09F918923882311F40C94A80388
:10074000ABEBB0E08C9182508C9381E0809362009F
:1007500000916200013011F00C94E4038EB5887FA3
:100760008EBD5A924A928091BB00A42DB52D8C93D8
:1007700081E00E944F2D5A924A928091C000A42D90
:10078000B52D8C9381E00E944F2D5A924A92809110
:10079000C100A42DB52D8C9381E00E944F2D0E94A5
:1007A0005E29269683E00E944B2DEBE0F0E0ABEB58
:1007B000B0E07BE70E94AE2F0091D000013011F035
:1007C0000C94E40381E08EBD0091D200023011F060
:1007D0000C9467044091C60000916000041718F063
:1007E00011F00C94F5030C946704809160008093E1
:1007F000C60000916000013011F00C940B0481E000
:1008000090E0A6EBB0E08D939C93ABE6B0E0E2E223
:10081000F0E60E94DA2D00916000023011F00C9495
:100820004F04A2EBB0E00D911C9141E050E0041B9D
:10083000150BA3E6B0E00D931C9302E010E00F93BC
:100840001F93A3E6B0E08D919C918A939A930E94A6
:100850007B2D2296402F512F1F910F91040F151FB2
:10086000A3E6B0E00D931C93A6EBB0E04D915C9134
:10087000A3E6B0E00D911C910417150711F40C9438
:100880001104A3E6B0E08D919C91A6EBB0E08D93AE
:100890009C93ABE6B0E0E2E2F0E60E94DA2D009134
:1008A0006000033011F00C945B04ABE6B0E0E4E2CE
:1008B000F0E60E94DA2D00916000043011F00C94F3
:1008C0006704ABE6B0E0E6E2F0E60E94DA2D00272E
:1008D000AAE6B0E08C9184FB0EF401E041E004173D
:1008E00081E009F080E08F930027A1EDB0E08C91CA
:1008F00087FB0EF401E041E0041781E009F080E09D
:100900009F9189238F930091D000013081E009F0FD
:1009100080E09F918923882311F40C94D204A6EBE4
:10092000B0E00D911C91013050E0150711F00C94CE
:10093000D204E0E6F0E0FA93EA930E94B81E229611
:1009400000916000003080E010F009F081E08F93AA
:10095000A2EBB0E04D915C91A0E6B0E00D911127C3
:100960000417150781E008F080E09F918923882310
:1009700011F40C94D204A0E6B0E00D91112741E0EF
:1009800050E0040F151FA6EBB0E00D931C93ABE6EF
:10099000B0E0E2E2F0E60E94DA2D70916A00706841
:1009A00070936A000027AAE6B0E08C9180FB0EF4F9
:1009B00001E040E0041711F00C949705E9E6F0E03F
:1009C000FA93EA930E94601E229600916900043017
:1009D00011F00C94F2040E94A20E70916A007068EB
:1009E00070936A0080E0809360000091690002309B
:1009F00081E009F080E08F930091BB00043681E034
:100A000008F080E09F918923882311F40C9410054D
:100A1000ABEBB0E08C918B5F8C9381E080936000B6
:100A200000916900033081E009F080E08F9300912C
:100A3000BB00053081E009F080E09F918923882385
:100A400011F40C94290581E08093BB0081E0809330
:100A5000600000916900033081E009F080E08F932D
:100A60000091BB00053080E010F009F081E09F911B
:100A70008923882311F40C944505ABEBB0E08C91ED
:100A800085508C9381E0809360000091600001307C
:100A900011F00C9486058EB5887F8EBD5A924A92CD
:100AA0008091BB00A42DB52D8C9381E00E944F2D29
:100AB0005A924A928091C000A42DB52D8C9381E06A
:100AC0000E944F2D5A924A928091C100A42DB52DBB
:100AD0008C9381E00E944F2D0E945E29269683E030
:100AE0000E944B2DEBE0F0E0ABEBB0E07BE70E9427
:100AF000AE2F0091D000013011F00C94810581E0FF
:100B00008EBD70916A00706870936A0000916900F0
:100B1000013011F00C949705ABE6B0E0E4E2F0E6AA
:100B20000E94DA2D70916A00706870936A00EBE69B
:100B3000F0E0ABE6B0E00E94CD2EABE6B0E08C91E9
:100B4000803081E009F480E08F93009169000030EB
:100B500081E009F480E09F91892B8F930091B80088
:100B6000013081E009F080E09F91892B882311F406
:100B70000C949E020091B800013011F00C94E10534
:100B800080E08093B800ABE6B0E0E4E2F0E60E94DB
:100B9000DA2D0027A1EDB0E08C9187FB0EF401E087
:100BA00041E0041711F00C94E10581E090E0A6EB20
:100BB000B0E08D939C93ABE6B0E0E2E2F0E60E94F9
:100BC000DA2DABE6B0E0E8E2F0E60E94D92F11F0B2
:100BD0000C941E0688EC8093BB008EB5887F8EBD7A
:100BE0005A924A928091BB00A42DB52D8C9381E03E
:100BF0000E944F2D5A924A928091C000A42DB52D8B
:100C00008C9381E00E944F2D5A924A928091C100AC
:100C1000A42DB52D8C9381E00E944F2D0E945E295A
:100C2000269683E00E944B2D0091D000013011F0F8
:100C30000C941C0681E08EBD0C94CD0CEAE2F0E62B
:100C40000E94D92F11F00C945C06EBE0F0E0ABEBC6
:100C5000B0E00E94BF2F8EB5887F8EBD5A924A9217
:100C60008091BB00A42DB52D8C9381E00E944F2D67
:100C70005A924A928091C000A42DB52D8C9381E0A8
:100C80000E944F2D5A924A928091C100A42DB52DF9
:100C90008C9381E00E944F2D0E945E29269683E06E
:100CA0000E944B2D0091D000013011F00C945A0697
:100CB00081E08EBD0C94CD0CECE2F0E60E94D92FC1
:100CC00011F00C94A4060E94E72DA0E6B0E08C93EE
:100CD00000916000003011F40C9463060E94EB2D2B
:100CE000A0ECB0E08C938EB5887F8EBD5A924A926C
:100CF0008091BB00A42DB52D8C9381E00E944F2DD7
:100D00005A924A928091C000A42DB52D8C9381E017
:100D10000E944F2D5A924A928091C100A42DB52D68
:100D20008C9381E00E944F2D0E945E29269683E0DD
:100D30000E944B2D0091D000013011F00C94A206BE
:100D400081E08EBD0C94CD0CEEE2F0E60E94D92F2E
:100D500011F00C94EC060E94E72DA0E6B0E08C9315
:100D600000916000003011F40C94AB060E94EB2D52
:100D7000A1ECB0E08C938EB5887F8EBD5A924A92DA
:100D80008091BB00A42DB52D8C9381E00E944F2D46
:100D90005A924A928091C000A42DB52D8C9381E087
:100DA0000E944F2D5A924A928091C100A42DB52DD8
:100DB0008C9381E00E944F2D0E945E29269683E04D
:100DC0000E944B2D0091D000013011F00C94EA06E6
:100DD00081E08EBD0C94CD0CE0E3F0E60E94D92FAB
:100DE00011F00C9431075A924A928091BE00A42DC2
:100DF000B52D8C9381E00E944F2D5A924A9280919A
:100E0000BF00A42DB52D8C9381E00E944F2D0E9430
:100E1000262A249682E00E944B2D0091C40041E0D6
:100E2000042BA0E6B0E00C937091D1007061709338
:100E3000D1008EB5887F8EBDEFE0F0E0A0E6B0E097
:100E40007BE70E94AE2F809160008093C4000091E8
:100E5000D000013011F00C942F0781E08EBD0C946E
:100E6000CD0CE2E3F0E60E94D92F11F00C94740748
:100E70005A924A9280E0A42DB52D8C9381E00E9475
:100E80004F2D5A924A9280E0A42DB52D8C9381E08B
:100E90000E944F2D0E94262A249682E00E944B2D0C
:100EA0000091C4004EEF0423A0E6B0E00C937091D3
:100EB000D1007F7E7093D1008EB5887F8EBDEFE02C
:100EC000F0E0A0E6B0E07BE70E94AE2F80916000EA
:100ED0008093C4000091D000013011F00C9472078F
:100EE00081E08EBD0C94CD0CE2E2F0E60E94D92F99
:100EF00011F00C94E4070091D000013011F00C9433
:100F000083070E94A20EA2EBB0E04D915C91A6EB8C
:100F1000B0E00D911C910417150718F011F00C9416
:100F2000DF070027A1EDB0E08C9186FB0EF401E015
:100F300040E0041711F00C94B007E6EBF0E0FA93F0
:100F4000EA935A924A9280E0A42DB52D8C9381E0C9
:100F50000E944F2D0E944B13249681E00E944B2D3E
:100F60000027A1EDB0E08C9186FB0EF401E041E09A
:100F7000041711F00C94DD070E94D10E0027A1ED9B
:100F8000B0E08C9186FB0EF401E040E0041711F014
:100F90000C94DD07E6EBF0E0FA93EA935A924A925A
:100FA00080E0A42DB52D8C9381E00E944F2D0E94EE
:100FB0004B13249681E00E944B2D0C94E20780E0B5
:100FC0008093C6000C94CD0CE4E3F0E60E94D92F88
:100FD00011F00C94F2070E94A20E80E08093C600EC
:100FE0000C94CD0CE6E3F0E60E94D92F11F00C949E
:100FF0002C080091D000013011F00C942A08002731
:10100000AAE6B0E08C9183FB0EF401E040E0041707
:1010100011F00C941C088EB5887F8EBD89B78B7F2C
:1010200089BF70916A00786070936A0084E690E0EE
:101030000E94B42E0C942A0870916A00777F7093F6
:101040006A0080E29EE49DBD8CBD81E08EBD89B7C3
:10105000846089BF0C94CD0CE4E2F0E60E94D92FA5
:1010600011F00C94C4080091D000013011F00C94E0
:101070003B080E94A20EA6EBB0E00E94622D002762
:10108000A1EDB0E08C9185FB0EF401E041E0041786
:1010900011F00C9460080027AAE6B0E08C9184FB64
:1010A0000EF401E040E0041711F00C945B08A6EB8D
:1010B000B0E00E94682D7091D1007F7D7093D100C7
:1010C000A2EBB0E04D915C91A6EBB0E00D911C91CC
:1010D0000417150718F011F00C9470080C9476089A
:1010E00081E090E0A6EBB0E08D939C930027A1ED0A
:1010F000B0E08C9186FB0EF401E040E0041711F0A3
:101100000C949508E6EBF0E0FA93EA935A924A922F
:1011100080E0A42DB52D8C9381E00E944F2D0E947C
:101120004B13249681E00E944B2D0027A1EDB0E0E7
:101130008C9186FB0EF401E041E0041711F00C9451
:10114000C2080E94D10E0027A1EDB0E08C9186FB71
:101150000EF401E040E0041711F00C94C208E6EB35
:10116000F0E0FA93EA935A924A9280E0A42DB52DCA
:101170008C9381E00E944F2D0E944B13249681E0B6
:101180000E944B2D0C94CD0CE6E2F0E60E94D92F84
:1011900011F00C943C090091D000013011F00C9436
:1011A000D3080E94A20EA6EBB0E00D911C91013075
:1011B00050E0150718F011F00C94E0080C94E608C4
:1011C000A6EBB0E00E94682D0C94EE08A2EBB0E014
:1011D0008D919C91A6EBB0E08D939C930027A1ED9F
:1011E000B0E08C9186FB0EF401E040E0041711F0B2
:1011F0000C940D09E6EBF0E0FA93EA935A924A92C6
:1012000080E0A42DB52D8C9381E00E944F2D0E948B
:101210004B13249681E00E944B2D0027A1EDB0E0F6
:101220008C9186FB0EF401E041E0041711F00C9460
:101230003A090E94D10E0027A1EDB0E08C9186FB07
:101240000EF401E040E0041711F00C943A09E6EBCB
:10125000F0E0FA93EA935A924A9280E0A42DB52DD9
:101260008C9381E00E944F2D0E944B13249681E0C5
:101270000E944B2D0C94CD0CE8E3F0E60E94D92F90
:1012800011F00C94AF09A6EBB0E00E94622DA2EB26
:10129000B0E04D915C91A6EBB0E00D911C9104176C
:1012A000150718F011F00C9457090C945D0981E0B2
:1012B00090E0A6EBB0E08D939C938EB5887F8EBDB9
:1012C000A2E7B0E00D911D912D913C91A2E9B0E013
:1012D0000D931D932D933C930027A1EDB0E08C91CD
:1012E00086FB0EF401E040E0041711F00C94A50910
:1012F0005A924A92A2E9B0E00D911D912D913C9134
:10130000A42DB52D0D931D932D933C9384E00E9445
:101310004F2D5A924A92A6EBB0E08D919C91A42D4C
:10132000B52D8D939C9382E00E944F2D5A924A9244
:1013300080E0A42DB52D8C9381E00E944F2D0E945A
:10134000AC16269687E00E944B2D0091D00001300C
:1013500011F00C94AD0981E08EBD0C94CD0CE8EF3A
:10136000FFE50E94D92F11F00C94230AA6EBB0E000
:101370000D911C91013050E0150718F011F00C94FC
:10138000C3090C94C909A6EBB0E00E94682D0C9427
:10139000D109A2EBB0E08D919C91A6EBB0E08D93CA
:1013A0009C938EB5887F8EBDA2E7B0E00D911D9114
:1013B0002D913C91A2E9B0E00D931D932D933C93A8
:1013C0000027A1EDB0E08C9186FB0EF401E040E037
:1013D000041711F00C94190A5A924A92A2E9B0E04B
:1013E0000D911D912D913C91A42DB52D0D931D9323
:1013F0002D933C9384E00E944F2D5A924A92A6EB83
:10140000B0E08D919C91A42DB52D8D939C9382E09D
:101410000E944F2D5A924A9280E0A42DB52D8C93B4
:1014200081E00E944F2D0E94AC16269687E00E9414
:101430004B2D0091D000013011F00C94210A81E075
:101440008EBD0C94CD0CEAE3F0E60E94D92F11F08A
:101450000C94330AECE0F0E0A6EBB0E07BE70E94EE
:10146000B02F0C94CD0CECE3F0E60E94D92F11F0D4
:101470000C94470A8DE181BD85E181BD0E94A20ED9
:1014800081B5886081BD0C94430A0C94CD0CABE609
:10149000B0E0EEE3F0E60E94D92F81E008F480E0AE
:1014A0008F93ABE6B0E0E0E4F0E60E94D92F81E054
:1014B00010F009F080E09F918923882311F40C94A7
:1014C0001B0B89B78B7F89BF8EB5887F8EBD0E942D
:1014D000E72DA0E6B0E08C9300916000003011F49D
:1014E0000C94670A0E94EB2DA6EBB0E08D93882741
:1014F0008C9380E08093D00070916A00777F709326
:101500006A00A2EBB0E04D915C91A6EBB0E00D91CA
:101510001C910417150780E010F009F081E08F930B
:10152000A6EBB0E00D911C91003050E0150781E072
:1015300009F080E09F91892B882311F40C94BB0A59
:1015400081E090E0A6EBB0E08D939C93E6EBF0E0B9
:10155000FA93EA935A924A9281E0A42DB52D8C9386
:1015600081E00E944F2D0E944B13249681E00E943F
:101570004B2D0C94190B0027A1EDB0E08C9186FB4C
:101580000EF401E040E0041781E009F080E08F9361
:10159000ABE6B0E0EEE3F0E60E94D92F81E009F07F
:1015A00080E09F918923882311F40C94EA0AE6EBEA
:1015B000F0E0FA93EA935A924A9281E0A42DB52D75
:1015C0008C9381E00E944F2D0E944B13249681E062
:1015D0000E944B2D0027A1EDB0E08C9186FB0EF40C
:1015E00001E040E0041781E009F080E08F93ABE672
:1015F000B0E0E0E4F0E60E94D92F81E009F080E05D
:101600009F918923882311F40C94190BE6EBF0E0E9
:10161000FA93EA935A924A9280E0A42DB52D8C93C6
:1016200081E00E944F2D0E944B13249681E00E947E
:101630004B2D0C94CD0CE2E4F0E60E94D92F11F072
:101640000C946A0B0E94E72DA0E6B0E08C93009109
:101650006000003011F40C94220B0E94EB2DABEBD8
:10166000B0E08C938EB5887F8EBD5A924A9280915D
:10167000BB00A42DB52D8C9381E00E944F2D5A9272
:101680004A928091C000A42DB52D8C9381E00E94D8
:101690004F2D5A924A928091C100A42DB52D8C9362
:1016A00081E00E944F2D0E945E29269683E00E94D1
:1016B0004B2DEBE0F0E0ABEBB0E07BE70E94AE2F10
:1016C0000091D000013011F00C94680B81E08EBDC8
:1016D0000C94CD0CE4E4F0E60E94D92F11F00C94A8
:1016E000B80B0E94E72DA0E6B0E08C93009160005B
:1016F000003011F40C94710B8091C3008093600052
:101700000E94EB2DA3ECB0E08C93A3ECB0E08C91A5
:101710008F738C930E940E0F0091C30040E104234D
:10172000A0E6B0E00C9300916000003111F00C9441
:101730009D0B0E940A0F0C949F0B0E940C0FA3ECB0
:10174000B0E08C918F7E8C938EB5887F8EBDEEE05D
:10175000F0E0A3ECB0E07BE70E94AE2F0091D00058
:10176000013011F00C94B60B81E08EBD0C94CD0CC1
:10177000E6EFFFE50E94D92F11F00C941C0C0091AC
:10178000C3004FE30423A0E6B0E00C930091D00027
:10179000013011F00C94D10BA0E6B0E08C91805890
:1017A0008C930027A1EDB0E08C9186FB0EF401E054
:1017B00041E0041711F00C94E20BA0E6B0E08C912C
:1017C000805C8C930027AAE6B0E08C9183FB0EF43A
:1017D00001E041E0041711F00C94F30BA0E6B0E037
:1017E0008C91805E8C938091B600809362008EB560
:1017F000887F8EBD31E0A0E6B0E00E94022E31E08D
:10180000ABEBB0E00E94022E31E0A2E6B0E00E9415
:10181000022E8091B2008093620031E0A2E6B0E037
:101820000E94022E0091D000013011F00C941A0C8D
:1018300081E08EBD0C94CD0CE6E4F0E60E94D92F39
:1018400011F00C949F0CA7EDB0E00D911D912D911E
:101850003C91A3EDB0E04D915D916D917C910E9422
:10186000202FA5E6B0E00D931D932D933D93A5E6A3
:10187000B0E00E94532DA5E6B0E00D911D912D9191
:101880003C9140E052E060E070E00E94142EA5E63A
:10189000B0E00D931D932D933D93A5E6B0E00D911F
:1018A0001D912D913C91A5ECB0E04C9155276627F8
:1018B00077270E94192EA5E6B0E04D935D936D93B6
:1018C0007D93A5E6B0E00D911D912D913C914AE0EC
:1018D00050E060E070E00E94192EA5E6B0E04D9364
:1018E0005D936D937D9344E150E060E070E0A5E688
:1018F000B0E00D911D912D913C910E94252F0CF48B
:1019000002C00C948D0C00E010E020E030E0A5E671
:10191000B0E00D931D932D933C938EB5887F8EBDC3
:1019200034E0A5E6B0E00E94022E0091D000013024
:1019300011F00C949D0C81E08EBD0C94CD0CE8E46C
:10194000F0E60E94D92F11F00C94B70C8EB5887F69
:101950008EBDA4EAB0E00E94F52D0091D0000130C8
:1019600011F00C94B50C81E08EBD0C94CD0CEAE422
:10197000F0E60E94D92F11F00C94CD0C8EB5887F23
:101980008EBD0E9448160091D000013011F00C94D9
:10199000CB0C81E08EBD0C94CD0C81E090E00E94D8
:1019A000B42E0027AAE6B0E08C9187FB0EF401E08C
:1019B00040E0041718F011F00C94E00C0C94990D11
:1019C00000916900003018F011F00C94E90C0C94AF
:1019D000500DA895E0E6F0E0FA93EA930E94601EAD
:1019E000229600916000043011F00C94440D0E9486
:1019F000A20E80E08093C6000E940C0F85E090E06C
:101A00000E94B42E80E080936200E0E6F0E0FA935A
:101A1000EA930E94601E2296A2E6B0E08C918F5F4E
:101A20008C9388E090E00E94B42E0091600000301A
:101A300081E009F080E08F9300916200043680E03D
:101A400010F009F081E09F91892B882311F40C9408
:101A5000050D00916200043618F011F00C94320D5F
:101A60000C94410D81B5886181BD877F81BDE3E61E
:101A7000F0E0FA93EA930E94C30F229681B5886042
:101A800081BD80E08093600081E090E00E94B42EF0
:101A900000916000003011F00C94E90C0C948F0D53
:101AA0000091D200013011F00C948B0D80E090E099
:101AB000A3E6B0E08D939C93E0E6F0E0FA93EA931E
:101AC0000E94B81E2296A3E6B0E00E94622DEF931A
:101AD000FF93ECE8F1E00E94882EFF91EF910091D6
:101AE0006000003081E009F080E08F93A3E6B0E071
:101AF0000D911C91083250E0150780E010F009F0BC
:101B000081E09F91892B882311F40C945C0D81E076
:101B100090E00E94B42E81E090E00E94B42E0091EB
:101B2000D000003011F00C94990D85E090E00E94F7
:101B3000B42E0C9499020F921F922F923F924F92C3
:101B40005F927F928F929F92AF92BF920F931F935B
:101B50002F933F934F935F936F937F938F939F93B5
:101B6000AF93BF93CF93DF93EF93FF938FB78F9391
:101B7000F89489B78B7F89BF8EB5887F8EBD5A92C6
:101B80004A9280E092E0A42DB52D8D939C9382E043
:101B90000E944F2D0E94C92C229682E00E944B2D5C
:101BA0000091DB000A3011F00C94D80D0E940A0F4E
:101BB0000E94A4250091DB000A3011F00C94E50D81
:101BC0000E940C0F80E08093DB00ABEDB0E08C91C5
:101BD0008F5F8C93A8950027A1EDB0E08C9186FBD8
:101BE0000EF401E040E0041711F00C940A0E5A9232
:101BF0004A9280E092E0A42DB52D8D939C9382E0D3
:101C00000E944F2D0E94C92C229682E00E944B2DEB
:101C10000E94A425A7EDB0E04D915D916D917C915E
:101C2000A3EDB0E00D911D912D913C910E94252FC7
:101C300080E00CF481E08F930027A1EDB0E08C915F
:101C400086FB0EF401E040E0041781E009F080E03B
:101C50009F918923882311F40C94390E80E49CE928
:101C60009DBD8CBD81E08EBD89B7846089BF0C9419
:101C7000820E80E08093D00070916A00777F70932D
:101C80006A000027A1EDB0E08C9186FB0EF401E024
:101C900040E0041711F00C94560EAAE6B0E08C91C7
:101CA00084FBA8EBB0E0882780F98C930091C300F7
:101CB0004FE70423A1E6B0E00C930E940C0F80E0F4
:101CC0008093C6000027A1EDB0E08C9183FB0EF459
:101CD00001E041E0041781E009F080E08F930027E4
:101CE000A1EDB0E08C9182FB0EF401E041E004171D
:101CF00081E009F080E09F91892B882311F40C94F6
:101D0000820EDC988F918FBFFF91EF91DF91CF9181
:101D1000BF91AF919F918F917F916F915F914F9103
:101D20003F912F911F910F91BF90AF909F908F90F7
:101D30007F905F904F903F902F901F900F9018953D
:101D4000F894FFCF89B78B7F89BF8EB5887F8EBD12
:101D500080E08093D00070916A00777F70936A0072
:101D60000027A1EDB0E08C9183FB0EF401E041E08F
:101D7000041781E009F080E08F930027A1EDB0E027
:101D80008C9182FB0EF401E041E0041781E009F040
:101D900080E09F91892B882311F40C94D00EDC985D
:101DA0000895DE9A6E98C498C598C7980E940C0F43
:101DB000E2E0F0E00E940E2EDE98C49A0E94A02E6F
:101DC00084E690E00E94B42EA8957091D1007F7BAC
:101DD0007093D100E0E6F0E0FA93EA930E9470225B
:101DE000229600916000003011F40C94070F70915E
:101DF000D10070647093D10084E690E00E94B42E0C
:101E0000DE9A6E98C498C598C7980C94090F0E94E2
:101E10009D150895AB980895AB9A089581E00E94AE
:101E2000C32E70916A007F7E70936A000091C30098
:101E300041E00423A881B9810C93A881B9810C9158
:101E4000003011F40C94290F70916A007061709346
:101E50006A007091D1007F777093D1000091C30028
:101E600042E00423A881B9810C93A881B9810C9127
:101E7000003011F40C94410F7091D1007068709390
:101E8000D10070916A007E7F70936A000091C30058
:101E900044E00423A881B9810C93A881B9810C91F5
:101EA000003011F40C94590F70916A0071607093B6
:101EB0006A0070916A007D7F70936A000091C30090
:101EC00048E00423A881B9810C93A881B9810C91C1
:101ED000003011F40C94710F70916A00726070936D
:101EE0006A0070916A007F7D70936A000091C30060
:101EF00040E20423A881B9810C93A881B9810C9197
:101F0000003011F40C94890F70916A007062709324
:101F10006A007091D1007F7E7093D1000091C4005F
:101F200041E00423A881B9810C93A881B9810C9167
:101F3000003011F40C94A10F7091D1007061709376
:101F4000D1000091C40046E00423A881B9810C931C
:101F5000A881B9810C9142E00E94C92F0C93A881FD
:101F6000B9818C918093D2000091D200033011F09E
:101F70000C94BD0F82E08093D20081E0481A88273C
:101F8000580A2296089582E00E94C32E81E00E94A2
:101F9000C32E81E00E94C32E80E0AA81BB818C9376
:101FA00083E4ACE9B0E08C938FE4ADE9B0E08C93CE
:101FB0008EE4AEE9B0E08C9386E4AFE9B0E08C93B8
:101FC00089E4A0EAB0E08C93AAE6B0E08C9185FBAE
:101FD000A881B981882780F98C9370916A0070621A
:101FE00070936A00A2E7B0E00D911D912D913C9194
:101FF000A2E9B0E00D931D932D933C935A924A921F
:10200000A2E9B0E00D911D912D913C91A42DB52D2B
:102010000D931D932D933C9384E00E944F2D5A9273
:102020004A9280E090E0A42DB52D8D939C9382E0A0
:102030000E944F2D5A924A9281E0A42DB52D8C9387
:1020400081E00E944F2D0E94AC16269687E00E94E8
:102050004B2D8FE00E94C32EE4EAF0E006E0A88159
:10206000B9810E94A02FA881B981ECE4F0E60E941A
:10207000D92F0FB68FE0481A8827580A22960FBE2C
:1020800081E009F080E08F9300918D00003181E0C4
:1020900009F080E09F918923882311F40C949E100D
:1020A00081E0AA81BB818C93A2E9B0E00D911D91E2
:1020B0002D913C91A2E7B0E00D931D932D933C939D
:1020C00070916A007F7D70936A005A924A92A2E9E9
:1020D000B0E00D911D912D913C91A42DB52D0D9346
:1020E0001D932D933C9384E00E944F2D5A924A9267
:1020F00080E090E0A42DB52D8D939C9382E00E940A
:102100004F2D5A924A9280E0A42DB52D8C9381E0F8
:102110000E944F2D0E94AC16269687E00E944B2D00
:10212000A2E9B0E00D911D912D913C91A2E7B0E0A4
:102130000D931D932D933C930E94F810A881B981B3
:102140008C9180FBAAE6B0E08C9185F98C93A6E790
:10215000B0E00D911D912D913C91A2E7B0E00D935F
:102160001D932D933C93A2E7B0E00D911D912D910D
:102170003C91A2E9B0E00D931D932D933C935A92AC
:102180004A92A2E9B0E00D911D912D913C91A42DB0
:10219000B52D0D931D932D933C9384E00E944F2DFC
:1021A0005A924A9280E090E0A42DB52D8D939C9395
:1021B00082E00E944F2D5A924A9280E0A42DB52DC4
:1021C0008C9381E00E944F2D0E94AC16269687E0EA
:1021D0000E944B2DAA81BB818C91AE81BF818D93D2
:1021E00088278C9384E0481A8827580A26960895F1
:1021F00082E00E94C32E81E00E94C32E81E00E94F3
:10220000C32E789481E090E0AC81BD818D939C9346
:10221000EA81FB81FA93EA93EE81FF81FA93EA93D4
:102220000E940E132496AA81BB810C91013011F0FB
:102230000C94251182E090E0AC81BD818D939C933C
:1022400081E08093C3000C944111023011F00C9492
:10225000341183E090E0AC81BD818D939C9380E04C
:102260008093C3000C944111033011F00C94411180
:1022700084E090E0AC81BD818D939C9383E080935A
:10228000C300EEE0F0E0A3ECB0E07BE70E94AE2FED
:10229000EC81FD81FA93EA935A924A9280E0A42D50
:1022A000B52D8C9381E00E944F2D0E944B132496F4
:1022B00081E00E944B2D0091D000003011F00C9471
:1022C0005B1188EC90E00E94B42E85E090E0AC8138
:1022D000BD818D939C93EA81FB81FA93EA93EE8111
:1022E000FF81FA93EA930E940E132496EEE0F0E049
:1022F000A3ECB0E00E94BF2FAA81BB810C910330F8
:1023000011F00C9485110C942212AA81BB810C91BE
:10231000013011F00C949311A3ECB0E08C91886023
:102320008C930C949C11023011F00C949C11A3EC32
:10233000B0E08C91877F8C93EEE0F0E0A3ECB0E00E
:102340007BE70E94AE2F88EC90E00E94B42E86E0DE
:1023500090E0AC81BD818D939C93EA81FB81FA93DF
:10236000EA93EE81FF81FA93EA930E940E1324967A
:10237000AA81BB810C91033011F00C94C1110C9413
:102380002212EEE0F0E0A3ECB0E00E94BF2FAA81A1
:10239000BB810C91013011F00C94D511A3ECB0E08D
:1023A0008C9184608C930C94DE11023011F00C94AB
:1023B000DE11A3ECB0E08C918B7F8C93EEE0F0E02B
:1023C000A3ECB0E07BE70E94AE2F88EC90E00E9487
:1023D000B42E87E090E0AC81BD818D939C93EA811F
:1023E000FB81FA93EA93EE81FF81FA93EA930E94CC
:1023F0000E132496EEE0F0E0A3ECB0E00E94BF2FB5
:10240000AA81BB810C91013011F00C940E12A3EC47
:10241000B0E08C9180628C930C941712023011F012
:102420000C941712A3ECB0E08C918F7D8C93EEE0AE
:10243000F0E0A3ECB0E07BE70E94AE2F88EC90E0E8
:102440000E94B42E88E090E0AC81BD818D939C9376
:10245000EC81FD81FA93EA930E94EC12229600919E
:10246000C30043E00423A881B9810C93A881B981FA
:102470000C91003011F00C94451283E090E0AC8197
:10248000BD818D939C930C945B12013011F00C94E0
:10249000511282E090E0AC81BD818D939C930C94AD
:1024A0005B12033011F00C945B1284E090E0AC817D
:1024B000BD818D939C93EC81FD81FA93EA930E94F8
:1024C000EC1222960091C30048E00423A881B98150
:1024D0000C93A881B9810C91003011F00C94781202
:1024E0008AE090E0AC81BD818D939C930C94821224
:1024F000083011F00C94821289E090E0AC81BD812B
:102500008D939C93EC81FD81FA93EA930E94EC12E7
:1025100022960091C30044E00423A881B9810C9362
:10252000A881B9810C91003011F00C949F128BE0BE
:1025300090E0AC81BD818D939C930C94A9120430E2
:1025400011F00C94A9128CE090E0AC81BD818D93C8
:102550009C93EC81FD81FA93EA930E94EC122296FF
:102560000091C30040E20423A881B9810C93A881A3
:10257000B9810C91003011F00C94C6128DE090E0FE
:10258000AC81BD818D939C930C94D012003211F0DC
:102590000C94D0128EE090E0AC81BD818D939C9321
:1025A000EC81FD81FA93EA930E94EC1222968FE06F
:1025B00090E0AC81BD818D939C93EC81FD81FA9379
:1025C000EA930E94EC1222960E940E0F84E0481AB1
:1025D0008827580A26960895E881F981FA93EA93A4
:1025E0005A924A9280E0A42DB52D8C9381E00E94EE
:1025F0004F2D0E944B13249681E00E944B2D82E3C5
:1026000090E00E94B42E0091D000003011F00C94A4
:10261000031382E390E00E94B42E089581E00E94AB
:10262000C32EEA81FB81FA93EA935A924A9280E0A0
:10263000A42DB52D8C9381E00E944F2D0E944B1349
:10264000249681E00E944B2D84E690E00E94B42EF7
:10265000E881F981FA93EA930E94601E2296A8818C
:10266000B9810C91003018F011F00C9439130C94CE
:1026700028130E94A20E84E190E00E94B42EA8814B
:10268000B9818C91AC81BD818C9381E0481A8827F7
:10269000580A2296089582E00E94C32E81E00E948B
:1026A000C32E8EB5887F8EBD70916A00777F709340
:1026B0006A00A2E7B0E00D911D912D913C91A2E935
:1026C000B0E00D931D932D933C935A924A92A2E948
:1026D000B0E00D911D912D913C91A42DB52D0D9340
:1026E0001D932D933C9384E00E944F2D5A924A9261
:1026F000AA85BB858D919C91A42DB52D8D939C931E
:1027000082E00E944F2D5A924A9280E0A42DB52D6E
:102710008C9381E00E944F2D0E94AC16269687E094
:102720000E944B2D40E050E060E070E0AEE8B0E089
:102730000D911D912D913C910E94252F11F00C942B
:10274000A3130C9497150E9412295A924A928091D1
:10275000BB00A42DB52D8C9381E00E944F2D5A9281
:102760004A928091C000A42DB52D8C9381E00E94E7
:102770004F2D5A924A928091C100A42DB52D8C9371
:1027800081E00E944F2D0E945E29269683E00E94E0
:102790004B2D5A924A92ACEBB0E08D919C91A42DB6
:1027A000B52D8D939C9382E00E944F2D0E94652A47
:1027B000229682E00E944B2D0027A1EDB0E08C9183
:1027C00084FB0EF401E041E0041711F00C940214B4
:1027D0005A924A928091BE00A42DB52D8C9381E02F
:1027E0000E944F2D5A924A928091BF00A42DB52D80
:1027F0008C9381E00E944F2D0E94262A249682E02D
:102800000E944B2DA2E9B0E00D911D912D913C91BC
:10281000A3EDB0E00D931D932D933C93A2E9B0E09E
:102820000D911D912D913C91AEE8B0E04D915D91DF
:102830006D917C910E941B2FA7EDB0E00D931D932D
:102840002D933D9380E0A881B9818C930E94A425AB
:1028500081E090E0AA81BB818D939C93AA81BB818A
:102860000D911C910F3F51E0150718F011F00C94D9
:102870006814AA81BB81AD90BC90ABEDB0E0AA0D0D
:10288000BB1D0C910F3F81E009F080E08F93AA817E
:10289000BB81AD90BC90ACEDB0E0AA0DBB1D0C911E
:1028A0000F3E80E010F009F081E09F91892388239A
:1028B00011F40C94611481E0A881B9818C930C947B
:1028C0006814AA81BB810E94622D11F00C942E1411
:1028D000A881B9810C91013011F00C942614AA81C1
:1028E000BB81AD90BC90ADEDB0E0AA0DBB1D8C914D
:1028F000AA81BB818D9388278C93AA81BB810D917E
:102900001C9140E150E00E94942DAA81BB814D931F
:102910005C9380E18093C500AA81BB810D911C91DD
:10292000013050E0150711F00C949B1484E0809363
:10293000C5000C942815023050E0150711F00C94D6
:10294000A61485E08093C5000C942815033050E050
:10295000150711F00C94B11486E08093C5000C9417
:102960002815043050E0150711F00C94BC1487E0D2
:102970008093C5000C942815053050E0150711F020
:102980000C94C71488E08093C5000C942815063079
:1029900050E0150711F00C94D2148AE08093C50022
:1029A0000C942815073050E0150711F00C94DD1435
:1029B0008CE08093C5000C942815083050E0150772
:1029C00011F00C94E8148EE08093C5000C94281547
:1029D000093050E0150711F00C94F31480E1809356
:1029E000C5000C9428150A3050E0150711F00C941E
:1029F000FE1484E18093C5000C9428150B3050E040
:102A0000150711F00C94091588E18093C5000C940A
:102A100028150C3050E0150711F00C9414158CE1BA
:102A20008093C5000C9428150D3050E0150711F067
:102A30000C941F1580E28093C5000C9428150E306D
:102A400050E0150711F00C94281588E28093C5001A
:102A5000AEE8B0E00D911D912D913C9140E052E027
:102A600060E070E00E94142EA5E6B0E00D931D9387
:102A70002D933D93A5E6B0E00D911D912D913C91D4
:102A8000A5ECB0E04C915527662777270E94192EB8
:102A9000A5E6B0E04D935D936D937D93A5E6B0E020
:102AA0000D911D912D913C9148EE53E060E070E056
:102AB0000E94192EA5E6B0E04D935D936D937D9332
:102AC000AC81BD810C91003011F00C94971581E020
:102AD0008093D00088EC9FEA9DBD8CBD89B784604F
:102AE00089BF81E08EBD0027A1EDB0E08C9183FB12
:102AF0000EF401E041E0041781E009F080E08F93DB
:102B00000027A1EDB0E08C9182FB0EF401E041E0E2
:102B1000041781E009F080E09F91892B882311F44C
:102B20000C949315DC9A85E090E00E94B42E83E02B
:102B3000481A8827580A24960895A895A2E7B0E075
:102B40000D911D912D913C91A6E7B0E00D931D9341
:102B50002D933C93A2E7B0E00D911D912D913C91F6
:102B6000A2E9B0E00D931D932D933C935A924A92A3
:102B7000A2E9B0E00D911D912D913C91A42DB52DB0
:102B80000D931D932D933C9384E00E944F2D5A92F8
:102B90004A9280E090E0A42DB52D8D939C9382E025
:102BA0000E944F2D5A924A9280E0A42DB52D8C930D
:102BB00081E00E944F2D0E94AC16269687E00E946D
:102BC0004B2DA895A2EBB0E00D911C91013050E087
:102BD000150710F00C9413165A924A9281E0A42D16
:102BE000B52D8C9381E00E944F2D0E94BF2A229622
:102BF00081E00E944B2D8CE291E00E94B42E5A920B
:102C00004A9280E0A42DB52D8C9381E00E944F2D37
:102C10000E94BF2A229681E00E944B2D7091D10024
:102C200070647093D100A895A2E7B0E00D911D915A
:102C30002D913C91A2E9B0E00D931D932D933C930F
:102C4000A6EBB0E00D911C91003050E0150781E03B
:102C500009F080E08F93A2EBB0E04D915C91A6EB80
:102C6000B0E00D911C910417150780E010F009F0F9
:102C700081E09F91892B882311F40C94451681E003
:102C800090E0A6EBB0E08D939C930E940C0F08950A
:102C900084E00E94C32EA3EDB0E00D911D912D9113
:102CA0003C91A881B9810D931D932D933C93A2E78C
:102CB000B0E00D911D912D913C91A2E9B0E00D93F2
:102CC0001D932D933C935A924A92A2E9B0E00D9144
:102CD0001D912D913C91A42DB52D0D931D932D93F8
:102CE0003C9384E00E944F2D5A924A928FE19EE4D9
:102CF000A42DB52D8D939C9382E00E944F2D5A9266
:102D00004A9280E0A42DB52D8C9381E00E944F2D36
:102D10000E94AC16269687E00E944B2DA2E7B0E0F9
:102D20000D911D912D913C91A2E9B0E00D931D9361
:102D30002D933C93A881B9810D911D912D913C91CA
:102D4000A3EDB0E00D931D932D933C9384E0481ABE
:102D50008827580A2296089581E00E94C32E81E0B8
:102D60000E94C32E81E00E94C32E80E090E0A4EB7D
:102D7000B0E08D939C9370916A007F7B70936A00A2
:102D800000E010E020E030E0AEE8B0E00D931D93ED
:102D90002D933C930027AAE6B0E08C9185FB0EF4BE
:102DA00001E041E0041781E009F080E08F93A885FD
:102DB000B9850D911C91003050E0150781E009F4B0
:102DC00080E09F9189238F93AE81BF810C91003069
:102DD00081E009F080E09F918923882311F40C940D
:102DE0004C17A6E9B0E0E885F9850E94382FE6E99E
:102DF000F0E0A8E6B7E00E94942FE8E6F7E0A6E945
:102E0000B0E01127222704E033270E94DD2E81E461
:102E1000AC81BD818C93AC81BD818C9180939C00F1
:102E200081E0E6E9F0E001E00A93ABE6B0E00E9461
:102E3000992FABE6B0E08C91ADE9B0E08C9382E0E5
:102E4000E6E9F0E001E00A93ABE6B0E00E94992FDA
:102E5000ABE6B0E08C91AEE9B0E08C9383E0E6E9BC
:102E6000F0E001E00A93ABE6B0E00E94992FABE6F8
:102E7000B0E08C91AFE9B0E08C9384E0E6E9F0E05B
:102E800001E00A93ABE6B0E00E94992FABE6B0E018
:102E90008C91A0EAB0E08C9389B78B7F89BF8EB507
:102EA000887F8EBD81B5886181BD877F81BDACEC97
:102EB000B0E00D911D912D913C91A8ECB0E00D93E7
:102EC0001D932D933C93A6E7B0E04D915D916D91DC
:102ED0007C91A2E7B0E00D911D912D913C910E9453
:102EE000252F11F00C947E1702E010E020E030E076
:102EF000A8ECB0E00D931D932D933C9380E0A88146
:102F0000B9818C93EA81FB81FA93EA935A924A92AF
:102F1000AE85BF850D911D912D913C91A42DB52DB0
:102F20000D931D932D933C9384E00E944F2D0E949E
:102F30009B27249684E00E944B2DAA81BB810C9193
:102F40000E3F11F40C94B0177091D100706470931F
:102F5000D10070916A00706470936A000C94C3177A
:102F60005A924A92AA85BB858D919C91A42DB52D2C
:102F70008D939C9382E00E944F2D0E94C41822964C
:102F800082E00E944B2DA881B9818C918F5F8C9338
:102F900040916F00A881B9810C91041781E009F07C
:102FA00080E08F930027AAE6B0E08C9186FB0EF4B8
:102FB00001E041E0041781E009F480E09F9189235A
:102FC000882311F40C94791800917E000B3011F0D5
:102FD0000C942618E8ECF0E0FA93EA935A924A929D
:102FE000A8ECB0E00D911D912D913C91A42DB52D33
:102FF0000D931D932D933C9384E00E944F2D0E94CE
:10300000041D249684E00E944B2DEA85FB85FA93EB
:10301000EA935A924A92A8ECB0E00D911D912D913D
:103020003C91A42DB52D0D931D932D933C9384E0DD
:103030000E944F2D0E949A1C249684E00E944B2DE2
:1030400080E0A881B9818C930C947718A6E7B0E052
:103050004D915D916D917C91A2E7B0E00D911D9134
:103060002D913C910E94252F11F00C943D18AA85BA
:10307000BB850E94532D0C947718E8ECF0E0FA938E
:10308000EA935A924A92A8ECB0E00D911D912D91CD
:103090003C91A42DB52D0D931D932D933C9384E06D
:1030A0000E944F2D0E94041D249684E00E944B2D07
:1030B000EA85FB85FA93EA935A924A92A8ECB0E02B
:1030C0000D911D912D913C91A42DB52D0D931D9326
:1030D0002D933C9384E00E944F2D0E949A1C2496CD
:1030E00084E00E944B2D80E0A881B9818C930C94E0
:1030F0007D18AA85BB850E94532D0027AAE6B0E063
:103100008C9186FB0EF401E041E0041711F00C9461
:103110008217C49AA885B9850D911C91003050E0A2
:10312000150711F00C949C18A4EBB0E08D919C91C4
:10313000A2EBB0E08D939C930091D000013081E030
:1031400009F080E08F930027A1EDB0E08C9186FB21
:103150000EF401E040E0041781E009F080E09F9167
:103160008923882311F40C94BE1880E593EC9DBD4F
:103170008CBD81E08EBD89B7846089BF83E0481A29
:103180008827580A2696089584E00E94C32E84E07A
:103190000E94C32E81E00E94C32E81E00E94C32EB4
:1031A00081E00E94C32E81E00E94C32E80E0AE81A8
:1031B000BF818C93AE81BF810C910F3018F011F05C
:1031C0000C94A71A81E0AC81BD818C93AC81BD8148
:1031D0000C910C3018F011F00C9406198FEF0E942E
:1031E000A72E0E94A92E0E94A82EAC81BD81AD9071
:1031F000BB24A0E8B0E0AA0DBB1D8C93AC81BD81BF
:103200008C918F5F8C9311F00C94E6188DE0AC815B
:10321000BD818C93AC81BD810C91043118F011F00B
:103220000C9424198FEF0E94A72E0E94A92E0E94B1
:10323000A82EA881B9818C93AC81BD818C918F5FC0
:103240008C9311F00C940A19EA85FB85FA93EA93A2
:10325000EA85FB85FA93EA930E942F1B24960027A8
:10326000AAE6B0E08C9186FB0EF401E041E0041781
:1032700011F00C943D190C949F1A80E0AA81BB8137
:103280008C9300918C00003281E009F080E08F93F4
:1032900000918C00003181E009F080E09F91892B42
:1032A000882311F40C94581981E0AA81BB818C9376
:1032B00000918100003081E009F480E08F9300915B
:1032C0008100053E81E009F480E09F9189238F937E
:1032D000AA81BB810C91013081E009F080E09F91CF
:1032E0008923882311F40C94941A00918C000032E5
:1032F00011F00C947F19A4EBB0E00E94622D00271E
:10330000AAE6B0E08C9185FB0EF401E040E00417E2
:1033100011F00C94B41981E0AC81BD818C93AC8523
:10332000BD854D915C91A4EBB0E00D911C9104170B
:10333000150781E009F080E08F93A4EBB0E00D91D8
:103340001C91003050E0150780E010F009F081E09A
:103350009F918923882311F40C94B21980E0AC81E9
:10336000BD818C930C94E81980E0AC81BD818C9375
:1033700081E0A881B9818C93A881B9810C91053035
:1033800018F011F00C94E819A881B981AD90BB2414
:10339000ABE9B0E0AA0DBB1D4C91A881B981AD90FD
:1033A000BB24A0E8B0E0AA0DBB1D0C91041711F4DA
:1033B0000C94E01981E0AC81BD818C930C94E819E8
:1033C000A881B9818C918F5F8C9311F00C94BC19FA
:1033D000AC81BD810C91003081E009F080E08F93D9
:1033E000AC85BD850D911C910F315EE4150781E020
:1033F00009F080E09F91892B882311F40C94941A92
:103400000E94C11AA885B9850D911D912D913C91FD
:1034100040E052E060E070E00E94192EAEE8B0E0BB
:103420004D935D936D937D93E2E9F0E0FA93EA9317
:103430005A924A92AE85BF850D911D912D913C9176
:10344000A42DB52D0D931D932D933C9384E00E94E4
:103450004F2D0E949A1C249684E00E944B2D80914F
:103460008C0080938D00AC85BD850D911C910F3132
:103470005EE4150711F00C94651AA8E6B7E0E4EBDA
:10348000F0E00E94382F0E94F32DE4E5F0E60E9460
:10349000FB2DA4EAB0E00E94F52DE4E5F0E60E94E1
:1034A000FB2D00918C00003111F00C945B1AE6E5C5
:1034B000F0E60E94FB2DA8E6B7E0E885F9850E94BA
:1034C0003B2F0E94F32D0E94072EAC81BD810C91F1
:1034D000003011F00C94941A70916A00706470932B
:1034E0006A0000918D00003181E009F080E08F9347
:1034F000AC85BD850D911C910F315EE4150781E00F
:1035000009F480E09F918923882311F40C94941A84
:10351000AA85BB850D911D912D913C91ACECB0E03D
:103520000D931D932D933C9300918100003011F079
:103530000C949F1A70916A00706470936A00AE8157
:10354000BF818C918F5F8C9311F00C94DA188FEF00
:103550000E94A72E0E94A92E0E94A82EA0E6B0E0ED
:103560008C938FEF0E94A72E0E94A92E0E94A82E56
:10357000A0E6B0E08C938CE0481A8827580A2C9675
:10358000089581E00E94C32EA4EAB0E088278C93BE
:1035900081E0A881B9818C93A881B9810C91083010
:1035A00018F011F00C94FB1AA881B981AD90BB24DE
:1035B000A0E8B0E0AA0DBB1D0C91003211F40C94F0
:1035C000F31AA881B981AD90BB24A0E8B0E0AA0DA0
:1035D000BB1D8C91A4EAB0E08F930E94E02D8F91E7
:1035E0008D9388278C93A881B9818C918F5F8C9360
:1035F00011F00C94CC1AA4EAB0E00E94E02DEAE5A8
:10360000F0E60E94DA2D89E0A881B9818C93A88127
:10361000B9810C910B3018F011F00C94291BA88182
:10362000B981AD90BB24A0E8B0E0AA0DBB1D8C9180
:10363000A4EAB0E08F930E94E02D8F918D938827AC
:103640008C93A881B9818C918F5F8C9311F00C942D
:10365000071B81E0481A8827580A2296089581E0BE
:103660000E94C32E81E00E94C32E84E00E94C32EDC
:103670008FEF0E94A72E0E94A92E0E94A82EAC8137
:10368000BD818C938FEF0E94A72E0E94A92E0E94CD
:10369000A82EAA81BB818C93AA81BB810C91112792
:1036A0002227332740E051E060E070E00E94142EB2
:1036B000A885B9850D931D932D933D93A885B98554
:1036C0000D911D912D913C91AC81BD814C9155275F
:1036D000662777270E941B2FA885B9850D931D9318
:1036E0002D933D93A885B9850D911D912D913C9108
:1036F00040E050E061E070E00E94142EA881B981A2
:103700000D931D932D933D938FEF0E94A72E0E9442
:10371000A92E0E94A82EAC81BD818C938FEF0E94B0
:10372000A72E0E94A92E0E94A82EAC81BD818C9349
:103730008FEF0E94A72E0E94A92E0E94A82EAC8176
:10374000BD818C938FEF0E94A72E0E94A92E0E940C
:10375000A82EAC81BD818C938FEF0E94A72E0E9472
:10376000A92E0E94A82EAC81BD818C938FEF0E9460
:10377000A72E0E94A92E0E94A82EAA81BB818C93FD
:10378000AA81BB810C9111272227332740E051E009
:1037900060E070E00E94142EA885B9850D931D93FA
:1037A0002D933D93A885B9850D911D912D913C9147
:1037B000AC81BD814C915527662777270E941B2F2E
:1037C000A885B9850D931D932D933D93A885B98543
:1037D0000D911D912D913C91A881B9814D915D91E3
:1037E0006D917C910E941B2FA885B9850D931D9327
:1037F0002D933D938FEF0E94A72E0E94A92E0E9429
:10380000A82EAC81BD818C938FEF0E94A72E0E94C1
:10381000A92E0E94A82EAA81BB818C93AA81BB816C
:103820000C9111272227332740E051E060E070E03F
:103830000E94142EA881B9810D931D932D933D9361
:10384000A881B9810D911D912D913C91AC81BD81D3
:103850004C915527662777270E941B2FA881B98195
:103860000D931D932D933D938FEF0E94A72E0E94E1
:10387000A92E0E94A82EAC81BD818C938FEF0E944F
:10388000A72E0E94A92E0E94A82EAA81BB818C93EC
:10389000AA81BB810C9111272227332740E051E0F8
:1038A00060E070E00E94142EAE81BF810D931D93E5
:1038B0002D933D93AE81BF810D911D912D913C9132
:1038C000AC81BD814C915527662777270E941B2F1D
:1038D000AE81BF810D931D932D933D93AE81BF812A
:1038E0000D911D912D913C9140E050E061E070E020
:1038F0000E94142EAE81BF810D931D932D933D9395
:10390000AE81BF810D911D912D913C91A881B9810E
:103910004D915D916D917C910E941B2FAE81BF8175
:103920000D931D932D933D9386E0481A8827580ADE
:103930002696089584E00E94C32E84E00E94C32E40
:10394000AC81BD810D911D912D913C9142E050E0E3
:1039500060E070E00E94202FA881B9810D931D9333
:103960002D933D93AFE6B0E00C911127222733272A
:10397000A881B9814D915D916D917C910E94142E29
:10398000AA81BB810D931D932D933D93AA81BB8189
:103990000D911D912D913C91A6E7B0E04D915D9167
:1039A0006D917C910E941B2FAA81BB810D931D9369
:1039B0002D933D9300917E000B3011F40C94F21C7A
:1039C000AA81BB810D911D912D913C9140E250E067
:1039D00060E070E00E941B2FAA81BB810D931D93B4
:1039E0002D933D93AA81BB810D911D912D913C9109
:1039F000AE81BF810D931D932D933C9388E0481AAF
:103A00008827580A2496089584E00E94C32E82E0F5
:103A10000E94C32E00917E000B3011F00C94481DC3
:103A2000AC81BD810D911D912D913C9140E850E0FC
:103A300060E070E00E94192EA3EDB0E04D935D931D
:103A40006D937D93AC81BD810D911C9140E850E058
:103A50000E94B42DA881B9810D931C93A881B981CE
:103A60000D911C9144E050E00E94CE2DA881B981B7
:103A70000D931C93A881B9810D911C9144E050E0F5
:103A8000040F151FA881B9810D931C930C947E1D02
:103A9000AC81BD810D911D912D913C9140E051E093
:103AA00060E070E00E94192EA3EDB0E04D935D93AD
:103AB0006D937D93AC81BD810D911C9140E051E0EF
:103AC0000E94B42DA881B9810D931C93A881B9815E
:103AD0000D911C9142E050E00E94CE2DA881B98149
:103AE0000D931C93A881B9810D911C9142E050E087
:103AF000040F151FA881B9810D931C93A3EDB0E0AD
:103B00000D911D912D913C91AAE7B0E04D915D91F1
:103B10006D917C910E941B2FA3EDB0E00D931D933E
:103B20002D933D93A3EDB0E00D911D912D913C910E
:103B3000ADE6B0E04D915C91662777270E941B2F80
:103B4000A3EDB0E00D931D932D933D930E94A4250A
:103B5000A881B981AD90BC90ABEDB0E0AA0DBB1DC2
:103B60008C91AA81BB818D9388278D938D938C93A3
:103B7000A881B9810E94682DAA81BB810D911D91F8
:103B80002D913C9140E051E060E070E00E94142EE5
:103B9000AA81BB810D931D932D933D93AA81BB8177
:103BA0000D911D912D913C91A881B981AD90BC9052
:103BB000ABEDB0E0AA0DBB1D4C91552766277727CA
:103BC0000E941B2FAA81BB810D931D932D933D93C2
:103BD00000917E000B3011F00C944E1EA881B9812B
:103BE0000E94682DAA81BB810D911D912D913C9160
:103BF00040E051E060E070E00E94142EAA81BB8199
:103C00000D931D932D933D93AA81BB810D911D9121
:103C10002D913C91A881B981AD90BC90ABEDB0E005
:103C2000AA0DBB1D4C915527662777270E941B2F95
:103C3000AA81BB810D931D932D933D93A881B981DA
:103C40000E94682DAA81BB810D911D912D913C91FF
:103C500040E051E060E070E00E94142EAA81BB8138
:103C60000D931D932D933D93AA81BB810D911D91C1
:103C70002D913C91A881B981AD90BC90ABEDB0E0A5
:103C8000AA0DBB1D4C915527662777270E941B2F35
:103C9000AA81BB810D931D932D933D93AA81BB8176
:103CA0000D911D912D913C91AE81BF810D931D937E
:103CB0002D933C9386E0481A8827580A2496089545
:103CC00080E0A881B9818C930027BB27A0E38C9169
:103CD00083FB0EF401E040E0041711F00C94741E15
:103CE00082E0A881B9818C930027BB27A0E38C9147
:103CF00084FB0EF401E040E0041711F00C94841EE4
:103D000081E0A881B9818C930027BB27A3E38C9124
:103D100081FB0EF401E040E0041711F00C94941EB6
:103D200083E0A881B9818C930027BB27A3E38C9102
:103D300081FB0EF401E040E0041781E009F080E02F
:103D40008F930027BB27A0E38C9183FB0EF401E047
:103D500040E0041781E009F080E09F9189238823E7
:103D600011F40C94B71E84E0A881B9818C93089556
:103D700081E00E94C32E81E00E94C32E82E00E9457
:103D8000C32E0027A1EDB0E08C9183FB0EF401E07F
:103D900041E0041711F00C94E31E80E0AC81BD817A
:103DA0008C930027BB27A9E38C9185FB0EF401E0DF
:103DB00040E0041711F00C94E11E81E0AC81BD815C
:103DC0008C930C947D1F5398549880E081BB909AFB
:103DD000919AEF93FF93E0EFF1E00E94882EFF911C
:103DE000EF9180E0AC81BD818C930027BB27A0E3DD
:103DF0008C9180FB0EF401E041E0041711F00C946B
:103E0000051F81E0AC81BD818C93AC81BD810C919B
:103E1000003018F011F00C940F1F0C94351F85E042
:103E200090E00E94B42E80E0AA81BB818C93002791
:103E3000BB27A0E38C9180FB0EF401E041E0041766
:103E400011F00C94271F81E0AA81BB818C93AA8179
:103E5000BB814C91AC81BD810C91041711F40C9481
:103E6000351F80E0AC81BD818C93AC81BD810C910C
:103E7000033011F00C94421F82E0AC81BD818C9321
:103E80000C94781FAC81BD810C91043081E008F462
:103E900080E08F93AC81BD810C91073081E010F000
:103EA00009F080E09F918923882311F40C945E1F10
:103EB00083E0AC81BD818C930C94781FAC81BD8173
:103EC0000C91083081E008F480E08F93AC81BD81D3
:103ED0000C910F3081E010F009F080E09F91892370
:103EE000882311F40C94781F84E0AC81BD818C93FD
:103EF00081E081BB9198539A549AAC81BD818C9199
:103F0000AE81BF818C9384E0481A8827580A269690
:103F1000089581E00E94C32E81E00E94C32EAC81EF
:103F2000BD818C91A881B9818C930E940A0F88EC85
:103F300090E00E94B42E5A924A9281E0A42DB52DB1
:103F40008C9381E00E944F2D0E94BF2A229681E02F
:103F50000E944B2DA895E9E6F0E0FA93EA930E94BF
:103F6000601E22968AE090E00E94B42E00916900C3
:103F7000003011F00C94AA1F86E990E00E94B42E44
:103F80005A924A9280E0A42DB52D8C9381E00E9434
:103F90004F2D0E94BF2A229681E00E944B2D84E67D
:103FA00090E00E94B42E5A924A9280E0A42DB52D42
:103FB0008C9381E00E944F2D0E94BF2A229681E0BF
:103FC0000E944B2DA895E9E6F0E0FA93EA930E944F
:103FD000601E22960E940C0F5A924A9281E0A42DF4
:103FE000B52D8C9381E00E944F2D0E94BF2A22960E
:103FF00081E00E944B2D84E690E00E94B42E5A92FC
:104000004A9280E0A42DB52D8C9381E00E944F2D23
:104010000E94BF2A229681E00E944B2D8AE090E008
:104020000E94B42E5A924A9280E0A42DB52D8C9312
:1040300081E00E944F2D0E94BF2A229681E00E94BB
:104040004B2D0E940A0F86E990E00E94B42E009149
:104050006900003018F011F00C9430200C94E21F2D
:1040600088E790E00E94B42E5A924A9281E0A42DF3
:10407000B52D8C9381E00E944F2D0E9451212296F4
:1040800081E00E944B2DA881B9810C91023011F082
:104090000C948A2000916900013011F00C94552095
:1040A00081E08093C3000C948320023011F00C94C3
:1040B0006D2080E08093C3005A924A9281E0A42D43
:1040C000B52D8C9381E00E944F2D0E9451212296A4
:1040D00081E00E944B2D0C948320033011F00C944E
:1040E000832083E08093C3005A924A9282E0A42DF9
:1040F000B52D8C9381E00E944F2D0E945121229674
:1041000081E00E944B2DEEE0F0E0A3ECB0E07BE715
:104110000E94AE2FA881B9810C91033011F00C944C
:10412000BD2000916900013011F00C949E20A4EC98
:10413000B0E08C9181608C930C94B620023011F029
:104140000C94B620A4ECB0E08C918E7F8C935A92A4
:104150004A9281E0A42DB52D8C9381E00E944F2DD1
:104160000E945121229681E00E944B2DEFE0F0E069
:10417000A4ECB0E07BE70E94AE2FA881B9810C913E
:10418000013011F00C940F2100916900013011F001
:104190000C94D620A4ECB0E08C9182608C93A4ECBB
:1041A000B0E08C918B7F8C930C940821023011F03D
:1041B0000C94F020A4ECB0E08C91897F8C935A92FF
:1041C0004A9281E0A42DB52D8C9381E00E944F2D61
:1041D0000E945121229681E00E944B2D0C940821CF
:1041E000033011F00C940821A4ECB0E08C918660AF
:1041F0008C935A924A9282E0A42DB52D8C9381E043
:104200000E944F2D0E945121229681E00E944B2D49
:10421000EFE0F0E0A4ECB0E07BE70E94AE2F0E945C
:104220000E0FA895E9E6F0E0FA93EA930E94601E6B
:10423000229685E090E00E94B42E00916900003043
:1042400011F00C94112186E990E00E94B42E5A924C
:104250004A9280E0A42DB52D8C9381E00E944F2DD1
:104260000E94BF2A229681E00E944B2D86E990E0B1
:104270000E94B42E5A924A9280E0A42DB52D8C93C0
:1042800081E00E944F2D0E94BF2A229681E00E9469
:104290004B2D0E940C0F82E0481A8827580A24965A
:1042A000089581E00E94C32E81E0A881B9818C939A
:1042B000AA81BB814C91A881B9810C91041718F097
:1042C00011F00C947E215A924A9282E0A42DB52DD1
:1042D0008C9381E00E944F2D0E94BF2A229681E09C
:1042E0000E944B2D8DE790E00E94B42EA881B981E9
:1042F0008C918F5F8C9311F00C94582181E0481AB7
:104300008827580A2296089581E00E94C32E81E0F2
:10431000A881B9818C93A881B9810C91063018F0DD
:1043200011F00C94A7210E940A0F8FE090E00E94E8
:10433000B42E0E940C0F84E690E00E94B42EA88157
:10434000B9818C918F5F8C9311F00C948B2181E05B
:10435000481A8827580A2296089580E08093C00062
:1043600080E08093C1000E94A02EC39A88EC90E068
:104370000E94B42E81B5886081BD0E9412295A9294
:104380004A9281E0A42DB52D8C9381E00E944F2D9F
:104390005A924A928091C000A42DB52D8C9381E051
:1043A0000E944F2D5A924A928091C100A42DB52DA2
:1043B0008C9381E00E944F2D0E945E29269683E017
:1043C0000E944B2D81B5886181BD877F81BD84E6C8
:1043D00090E00E94B42EFF27E0E1FA93EA935A920C
:1043E0004A928BE0A42DB52D8C9381E00E944F2D35
:1043F0000E94552C249681E00E944B2D013051E003
:10440000150711F00C941D225A924A92ACEBB0E0C1
:104410008D919C91A42DB52D8D939C9382E00E944B
:104420004F2D0E94652A229682E00E944B2DECE5DA
:10443000F0E60E94FB2D0E94072E5A924A9282E3D8
:10444000A42DB52D8C9381E00E944F2D5A924A9253
:104450008091C000A42DB52D8C9381E00E944F2D3A
:104460005A924A928091C100A42DB52D8C9381E07F
:104470000E944F2D0E945E29269683E00E944B2DBC
:10448000C29AD89A82E390E00E94B42E089581E007
:104490000E94C32E81E00E94C32E8FEFAA81BB81B0
:1044A0008C9380E0A881B9818C93A881B9810C910B
:1044B000073018F011F00C946A2291E0AA81BB81B8
:1044C0000E94962EA881B9818C918F5F8C9311F0F8
:1044D0000C94552282E0481A8827580A2496089599
:1044E00081E00E94C32E81E00E94C32E81E00E94E1
:1044F000C32E82E00E94C32E82E00E94C32E8FEF63
:10450000AA85BB858C9381E0A885B9858C93A88505
:10451000B9850C91003418F011F00C9499220E9486
:104520004722A885B9858C918F5F8C9311F00C94EC
:104530008722C49881E0A885B9858C93A885B98520
:104540000C91003418F011F00C94B0220E94472214
:10455000A885B9858C918F5F8C9311F00C949E2265
:104560008AE090E00E94B42EA895EE81FF81FA9334
:10457000EA935A924A9280E4A42DB52D8C9381E05F
:104580000E944F2D5A924A9200E010E020E030E065
:10459000A42DB52D0D931D932D933C9384E00E9483
:1045A0004F2D0E948128269685E00E944B2DAE81DA
:1045B000BF810C91013011F40C94E722C49AE0E61B
:1045C000F0E60E94FB2D0E94072E0C949E2581E0B0
:1045D000AA85BB858C93A89580E090E0A881B981DD
:1045E0008D939C93EE81FF81FA93EA935A924A92BB
:1045F00081E4A42DB52D8C9381E00E944F2D5A9219
:104600004A9200E010E020E030E0A42DB52D0D939B
:104610001D932D933C9384E00E944F2D0E9481288E
:10462000269685E00E944B2DA881B9810E94622DBB
:10463000AE81BF810C91003081E009F080E08F9362
:10464000A881B9810D911C91003050E0150781E0DF
:1046500009F080E09F91892B882311F40C94F222B9
:10466000C49AA881B9810D911C91003050E01507C2
:1046700011F00C944323E8E6F0E60E94FB2D0E9423
:10468000072E0C949E25A89584E690E00E94B42EF7
:10469000A895C49881E090E00E94B42EEE81FF813D
:1046A000FA93EA935A924A9280E5A42DB52D8C9301
:1046B00081E00E944F2D5A924A9201E010E020E0E2
:1046C00030E0A42DB52D0D931D932D933C9384E0E4
:1046D0000E944F2D0E948128269685E00E944B2D36
:1046E00085E090E00E94B42EC49A8AE090E00E9497
:1046F000B42EA89500E010E020E030E0AAE7B0E09A
:104700000D931D932D933C9300E010E020E030E0EA
:10471000A3EDB0E00D931D932D933C930E94A4252F
:1047200000E010E020E030E0A3EDB0E00D931D9339
:104730002D933C930027A1EDB0E08C9186FB0EF405
:1047400001E041E0041711F00C94A8230C949E257D
:10475000A8950091E800023011F40C943C2480915B
:104760009E0280937E00A5EAB2E00D91112740E001
:1047700051E00E94CE2DAA81BB810D931C93AA818A
:10478000BB810D911C91A4EAB2E04D915527040F15
:10479000151FAA81BB810D931C93AA81BB810D912A
:1047A0001C912227332740E050E061E070E00E9436
:1047B000142EAAE7B0E00D931D932D933D93A3EA29
:1047C000B2E00D91112740E051E00E94CE2DAA8168
:1047D000BB810D931C93AA81BB810D911C91A2EA10
:1047E000B2E04D915527040F151FAA81BB810D938F
:1047F0001C93AAE7B0E00D911D912D913C91AA81E7
:10480000BB814D915C91662777270E941B2FAAE7F9
:10481000B0E00D931D932D933D9300917E000C30DD
:1048200011F00C9416248BE080937E0000917E00A2
:104830000E3011F00C941F248BE080937E000091C9
:104840007E000F3011F00C9428248BE080937E00C2
:10485000AAE7B0E00D911D912D913C91A3EDB0E040
:104860000D931D932D933C930E94A425A3EDB0E0DE
:104870000E946E2D0C94902400911201063411F0C8
:104880000C94662484E080937E0087E3A885B98534
:104890008C93A885B9850C910C3318F011F00C9409
:1048A0006424A885B985AD90BB24ABEDB0E0AA0D1A
:1048B000BB1D8C910E940A2EA885B9858C918F5FB3
:1048C0008C9311F00C9449240E94072E00912E0124
:1048D000063411F00C9490248BE080937E0083E5E5
:1048E000A885B9858C93A885B9850C91073518F0F2
:1048F00011F00C948E24A885B985AD90BB24ABED46
:10490000B0E0AA0DBB1D8C910E940A2EA885B98526
:104910008C918F5F8C9311F00C9473240E94072E5E
:10492000E2E7F0E60E94FB2DA8E6B7E0EEE7F0E054
:104930000E94472F0E94F32D0E94072EE4E8F0E624
:104940000E94FB2DA8E6B7E0EAE7F0E00E943B2FCB
:104950000E94F32D0E94072E84E0A885B9858C93D0
:10496000A885B9850C910B3018F011F00C94CB246C
:10497000A885B985AD90BB24ABEDB0E0AA0DBB1DF9
:104980008C910E940A2EA885B9858C918F5F8C939B
:1049900011F00C94B0240E94072E8091E9008093BE
:1049A0006F00E6E9F0E60E94FB2DA8E6B7E0EFE62F
:1049B000F0E00E94472F0E94F32D0E94072E0091E5
:1049C0006F00003011F00C94E7240C949E250091A8
:1049D0006F00003418F011F00C94F0240C94F224C1
:1049E0000C949E258091EA00AE81BF818C938091CA
:1049F000EB00AC81BD818C93AC81BD819C91AE817B
:104A0000BF818C91ADE6B0E08D939C938091F200D4
:104A1000AE81BF818C938091F300AC81BD818C937A
:104A2000AC81BD819C91AE81BF818C91A0E7B0E04B
:104A30008D939C93A0E7B0E00D911C91003050E065
:104A4000150711F00C943A2580910001AE81BF81C9
:104A50008C9380910101AC81BD818C93AC81BD812F
:104A60009C91AE81BF818C91A0E7B0E08D939C9327
:104A70000C943A25A0E7B0E00D911C91003050E075
:104A8000150711F00C9446250C949E2502E010E0C9
:104A900020E030E0A0E7B0E04D915C9166277727F9
:104AA0000E94142EA2E7B0E00D931D932D933D9329
:104AB000A2E7B0E00D911D912D913C91ADE6B0E0E3
:104AC0004D915C91662777270E941B2FA2E7B0E0EB
:104AD0000D931D932D933D93A2E7B0E00D911D9191
:104AE0002D913C91A3EDB0E04D915D916D917C9144
:104AF0000E941B2FA2E7B0E00D931D932D933D93D1
:104B0000E6EAF0E60E94FB2DA8E6B7E0E2E7F0E077
:104B10000E943B2F0E94F32D0E94072EA2E7B0E0D7
:104B20000D911D912D913C91A3EDB0E00D931D933E
:104B30002D933C9380E0AA85BB858C9387E0481A2F
:104B40008827580A2A96089581E00E94C32E81E0A2
:104B50000E94C32E82E00E94C32E82E00E94C32ED8
:104B60008FEFAE81BF818C9391E0AE81BF810E94B7
:104B7000962E91E0AE81BF810E94962E91E0AE818B
:104B8000BF810E94962E91E0AE81BF810E94962E39
:104B900091E0AE81BF810E94962E91E0AE81BF81EF
:104BA0000E94962E91E0AE81BF810E94962E91E0E8
:104BB000AE81BF810E94962E91E0AE81BF810E949E
:104BC000962E91E0AE81BF810E94962E91E0AE813B
:104BD000BF810E94962E91E0AE81BF810E94962EE9
:104BE00091E0AE81BF810E94962E91E0AE81BF819F
:104BF0000E94962E91E0AE81BF810E94962E91E098
:104C0000AE81BF810E94962EC49880E090E0A8817A
:104C1000B9818D939C938FEF0E94A72E0E94A92E9D
:104C20000E94A82EAE81BF818C93A881B9810E9479
:104C3000622DAE81BF810C91003081E009F480E0EB
:104C40008F93A881B9810D911C91003050E0150718
:104C500081E009F080E09F91892B882311F40C9466
:104C60000B26A881B9810D911C91003050E01507E9
:104C700011F00C944826EEEAF0E60E94FB2D0E940B
:104C8000072E7091D10070647093D1000C94952719
:104C9000EE81FF81FA93EA935A924A9281E5A42D1C
:104CA000B52D8C9381E00E944F2D5A924A92A3ED2C
:104CB000B0E00D911D912D913C91A42DB52D0D933A
:104CC0001D932D933C9384E00E944F2D0E948128D8
:104CD000269685E00E944B2D0027A1EDB0E08C9137
:104CE00086FB0EF401E041E0041711F00C948826D5
:104CF000ECEBF0E60E94FB2DA8E6B7E0E3EDF0E078
:104D00000E943B2F0E94F32D0E94072E0C949527A2
:104D1000A895AE81BF810C91003011F00C94D32680
:104D200080E090E0A881B9818D939C938FEF0E94E1
:104D3000A72E0E94A92E0E94A82EAE81BF818C931F
:104D4000A881B9810E94622DAE81BF810C91003093
:104D500081E009F480E08F93A881B9810D911C91C5
:104D6000003050E0150781E009F080E09F91892B29
:104D7000882311F40C949626A881B9810D911C9179
:104D8000003050E0150711F00C94D326E6EDF0E664
:104D90000E94FB2D0E94072E7091D10070647093C9
:104DA000D1000C949527AE81BF810C910F3F11F07B
:104DB0000C941D2780E090E0A881B9818D939C938D
:104DC0008FEF0E94A72E0E94A92E0E94A82EAE81CE
:104DD000BF818C93A881B9810E94622DAE81BF8171
:104DE0000C910F3F81E009F480E08F93A881B98195
:104DF0000D911C91003050E0150781E009F080E032
:104E00009F91892B882311F40C94E026A881B98105
:104E10000D911C91003050E0150711F00C941D27E6
:104E2000E4EEF0E60E94FB2D0E94072E7091D10067
:104E300070647093D1000C949527AE81BF810C9162
:104E40000E3F11F40C943A27E2EFF0E60E94FB2D9E
:104E5000A8E6B7E0EE81FF810E94472F0E94F32D64
:104E60000E94072EC49A7091D10070647093D10093
:104E70000C94952780E090E0AA81BB818D939C9350
:104E800080E0AE81BF818C93AE81BF810C910F3FDA
:104E900018F011F00C947C27AA81BB810E94622D2E
:104EA0008FEF0E94A72E0E94A92E0E94A82EAA81F1
:104EB000BB81AD90BC90ABEDB0E0AA0DBB1D8C9357
:104EC000AA81BB810E94622D8FEF0E94A72E0E94B3
:104ED000A92E0E94A82EAA81BB81AD90BC90ABEDFB
:104EE000B0E0AA0DBB1D8C93AE81BF818C918F5F0A
:104EF0008C9311F00C9444278FEF0E94A72E0E94F0
:104F0000A92E0E94A82EAE81BF818C938FEF0E94A4
:104F1000A72E0E94A92E0E94A82EAE81BF818C933D
:104F2000C49AA3EDB0E00E94532D86E0481A88276A
:104F3000580A2896089582E00E94C32E81E00E94BC
:104F4000C32E80E0AE81BF818C930E944722C4981B
:104F500080E090E0AA81BB818D939C938FEF0E94AB
:104F6000A72E0E94A92E0E94A82EA881B9818C93F9
:104F7000AA81BB810E94622DA881B9810C91003069
:104F800081E009F480E08F93AA81BB810D911C918F
:104F9000003050E0150781E009F080E09F91892BF7
:104FA000882311F40C94AE27AA81BB810D911C912A
:104FB000003050E0150711F00C94EB27EEEAF0E614
:104FC0000E94FB2D0E94072E7091D1007064709397
:104FD000D1000C947B28E881F981FA93EA935A92E4
:104FE0004A9281E5A42DB52D8C9381E00E944F2D2E
:104FF0005A924A92AA85BB850D911D912D913C91A3
:10500000A42DB52D0D931D932D933C9384E00E9408
:105010004F2D0E948128269685E00E944B2DA88165
:10502000B9810C91003011F00C94422880E090E09E
:10503000AA81BB818D939C938FEF0E94A72E0E9423
:10504000A92E0E94A82EA881B9818C93AA81BB8128
:105050000E94622DA881B9810C91003081E009F491
:1050600080E08F93AA81BB810D911C91003050E0AC
:10507000150781E009F080E09F91892B882311F4C6
:105080000C941C28A881B9810C910F3F11F00C944D
:10509000752880E090E0AA81BB818D939C938FEF6F
:1050A0000E94A72E0E94A92E0E94A82EA881B98135
:1050B0008C93AA81BB810E94622DA881B9810C9139
:1050C0000F3F81E009F480E08F93AA81BB810D91AD
:1050D0001C91003050E0150781E009F080E09F91BD
:1050E000892B882311F40C944F28A881B9818C91C5
:1050F000AE81BF818C9383E0481A8827580A249692
:10510000089584E00E94C32E81E00E94C32E82E0B5
:105110000E94C32E8FEFAA81BB818C9391E0AA815C
:10512000BB810E94962E91E0A885B9850E94962E9B
:10513000AE81BF810D911D912D913C9140E052E0D7
:1051400060E070E00E94142EAC81BD810D931D9330
:105150002D933D93AC81BD818F9314968E910E94C7
:1051600007298E910E9407298E910E9407298E910E
:105170000E94072985E90E9407298F9180E090E02D
:10518000A881B9818D939C938FEF0E94A72E0E94D6
:10519000A92E0E94A82EAA81BB818C93A881B981D7
:1051A0000E94622DAA81BB810C910F3F81E009F41E
:1051B00080E08F93A881B9810D911C91003050E05F
:1051C000150781E009F080E09F91892B882311F475
:1051D0000C94C428A881B9810D911C91003050E035
:1051E000150711F00C94FF28E0E0F1E60E94FB2D7A
:1051F0000E94072E7091D10070647093D100AA8133
:10520000BB818C91AA85BB858C930C940C298FB99A
:10521000779BFECF8FB1089587E0481A8827580AF8
:10522000269608955A924A9284E298E0A42DB52DCC
:105230008D939C9382E00E944F2D5A924A9280E077
:10524000A42DB52D8C9381E00E944F2D0E94FA2B46
:10525000249683E00E944B2DEF93FF93ECE8F1E05E
:105260000E94882EFF91EF91BB27A0E38C9182FBD7
:10527000DEF789E190E00E94B42E5A924A9280E2D1
:1052800098E0A42DB52D8D939C9382E00E944F2D24
:105290005A924A9280E0A42DB52D8C9381E00E9411
:1052A0004F2D0E94FA2B249683E00E944B2D89E11A
:1052B00090E00E94B42E0E94822A089582E00E940B
:1052C000C32E82E00E94C32E82E00E94C32EA885D6
:1052D000B9850C91003081E009F080E08F93AE81B8
:1052E000BF810C91003081E009F080E09F9189231B
:1052F000882311F40C948E29AA85BB858C91AA81F0
:10530000BB818D9388278C93AA85BB858C91A881BE
:10531000B9818D9388278C930C94D029AA85BB855D
:105320000D911127A885B9854D915527040F151F9B
:10533000AA81BB810D931C93AA81BB810D911C9105
:105340000F3F50E0150718F011F00C94A9290C94A8
:10535000AF298FEF90E0AA81BB818D939C93AA85A2
:10536000BB850D911127AE81BF814D915527040F4B
:10537000151FA881B9810D931C93A881B9810D9146
:105380001C910F3F50E0150718F011F00C94CA293A
:105390000C94D0298FEF90E0A881B9818D939C93D4
:1053A00000E011E0AA81BB814D915C910E94CE2D5D
:1053B000AC81BD810D931C93AC81BD810D911C917D
:1053C000A881B9814D915C91040F151FAC81BD81FD
:1053D0000D931C935A924A92AE81BF818D919C91FC
:1053E000A42DB52D8D939C9382E00E944F2D5A924F
:1053F0004A928BE0A42DB52D8C9381E00E944F2D15
:105400000E94FA2B249683E00E944B2D5A924A92D6
:1054100080E298E0A42DB52D8D939C9382E00E94AC
:105420004F2D5A924A9280E0A42DB52D8C9381E0A5
:105430000E944F2D0E94FA2B249683E00E944B2D50
:1054400086E0481A8827580A2696089582E00E9426
:10545000C32E00E110E0AC81BD814D9155270E9423
:10546000CE2DA881B9810D931C93A881B9810D918E
:105470001C91AA81BB814D915527040F151FA8814E
:10548000B9810D931C935A924A92AA81BB818D9146
:105490009C91A42DB52D8D939C9382E00E944F2D5D
:1054A0005A924A9282E0A42DB52D8C9381E00E94FD
:1054B0004F2D0E94FA2B249683E00E944B2D82E010
:1054C000481A8827580A229608955A924A92AA8121
:1054D000BB818D919C91A42DB52D8D939C9382E0E1
:1054E0000E944F2D5A924A9283E0A42DB52D8C93A1
:1054F00081E00E944F2D0E94FA2B249683E00E94A7
:105500004B2D089581E00E94C32E81E00E94C32E9E
:10551000C49AD898C29880E0A881B9818C9380E021
:10552000AA81BB818C93AA81BB810C910F3118F0A9
:1055300011F00C94B72A91E0A881B9810E94962EAF
:1055400091E0A881B9810E94962E91E0A881B9814D
:105550000E94962E91E0A881B9810E94962EAA8180
:10556000BB818C918F5F8C9311F00C94932AC29A1B
:10557000D89A82E0481A8827580A2496089581E02C
:105580000E94C32E5A924A9280E298E0A42DB52D33
:105590008D939C9382E00E944F2D5A924A9280E014
:1055A000A42DB52D8C9381E00E944F2D0E94FA2BE3
:1055B000249683E00E944B2DAA81BB810C91003080
:1055C00011F00C94F22A5A924A9280E0A42DB52D43
:1055D0008C9381E00E944F2D0E946C2B229681E0DB
:1055E0000E944B2DAA81BB810C91013011F00C94CB
:1055F000082B5A924A9285E6A42DB52D8C9381E012
:105600000E944F2D0E946C2B229681E00E944B2D10
:10561000AA81BB810C91023011F00C94352B5A9267
:105620004A9283E6A42DB52D8C9381E00E944F2DE4
:105630000E946C2B229681E00E944B2D88EC90E01A
:105640000E94B42E5A924A9280E0A42DB52D8C93DC
:1056500081E00E944F2D0E946C2B229681E00E94D7
:105660004B2D82E390E00E94B42EAA81BB810C9165
:10567000033011F00C945E2B5A924A9282E6A42DCC
:10568000B52D8C9381E00E944F2D0E946C2B2296A9
:1056900081E00E944B2D80E991E00E94B42E5A9245
:1056A0004A9280E0A42DB52D8C9381E00E944F2D6D
:1056B0000E946C2B229681E00E944B2D8AE090E0A4
:1056C0000E94B42E8AE090E00E94B42E81E0481A35
:1056D0008827580A2296089581E00E94C32EC49A12
:1056E000D898C298AA81BB810C91003018F011F0B3
:1056F0000C947C2B0C94B62B83E5A881B9818C93F8
:1057000091E0A881B9810E94962E8FEEA881B9817F
:105710008C9391E0A881B9810E94962E8EE6A88193
:10572000B9818C9391E0A881B9810E94962E91E075
:10573000AA81BB810E94962E80E0A881B9818C93BA
:1057400091E0A881B9810E94962E91E0A881B9814B
:105750000E94962E91E0A881B9810E94962E91E038
:10576000A881B9810E94962E0C94F22B85E4A88121
:10577000B9818C9391E0A881B9810E94962E88E727
:10578000A881B9818C9391E0A881B9810E94962E5D
:1057900089E6A881B9818C9391E0A881B9810E94A2
:1057A000962E84E7A881B9818C9391E0A881B98174
:1057B0000E94962E80E0A881B9818C9391E0A88107
:1057C000B9810E94962E91E0A881B9810E94962EFF
:1057D00091E0A881B9810E94962E91E0A881B981BB
:1057E0000E94962EC29AD89A81E0481A8827580AB1
:1057F0002296089581E00E94C32EC29AD8985A92A8
:105800004A9282E0A42DB52D8C9381E00E944F2D09
:105810000E94AF2C229681E00E944B2D5A924A9210
:10582000AC81BD818C91A42DB52D8C9381E00E941B
:105830004F2D0E94AF2C229681E00E944B2DAC810F
:10584000BD8111968C91A881B9818C935A924A920C
:10585000AA81BB818C91A42DB52D8C9381E00E94EF
:105860004F2D0E94AF2C229681E00E944B2DAC81DF
:10587000BD818C91A881B9818C935A924A92AA8158
:10588000BB818C91A42DB52D8C9381E00E944F2D6E
:105890000E94AF2C229681E00E944B2DD89A81E085
:1058A000481A8827580A2296089581E00E94C32E3C
:1058B00081E00E94C32E82E00E94C32EC29AD89833
:1058C0005A924A9283E0A42DB52D8C9381E00E94D8
:1058D0004F2D0E94AF2C229681E00E944B2D5A92B0
:1058E0004A92A885B9858C91A42DB52D8C9381E021
:1058F0000E944F2D0E94AF2C229681E00E944B2DDA
:10590000EC81FD81FA93EA930E94B52C2296EA81FC
:10591000FB81FA93EA930E94B52C2296D89AAC8127
:10592000BD810D91112740E051E00E94CE2DA8814C
:10593000B9810D931C93A881B9810D911C91AA8105
:10594000BB814D915527040F151FA885B9850D936F
:105950001C9384E0481A8827580A2696089591E0F7
:10596000A881B9810E94962E089581E00E94C32EDD
:1059700091E0A881B9810E948B2EA881B9818C9178
:10598000AA81BB818C9381E0481A8827580A229605
:10599000089582E00E94C32E81E00E94C32EC49A23
:1059A000BB27A0E38C9182FBDEF7C298AC81BD815E
:1059B0000D911C91003052E0150711F00C94182D38
:1059C00081E090E0AA81BB818D939C9380E0A881C7
:1059D000B9818C93A881B9810C910F3018F011F026
:1059E0000C94162DBB27A0E38C9182FBDEF790E28E
:1059F000AA81BB81AD90BC90ABEDB0E0AA0DBB1D00
:105A00000E94962EAA81BB810D911C9140E250E02C
:105A1000040F151FAA81BB810D931C93A881B98126
:105A20008C918F5F8C9311F00C94EA2C0C94442D84
:105A300081E090E0AA81BB818D939C93AC81BD8174
:105A40004D915C91AA81BB810D911C9104171507A2
:105A500018F011F00C94442DBB27A0E38C9182FB2D
:105A6000DEF7C29A91E0AA81BB81AD90BC90ABED0C
:105A7000B0E0AA0DBB1D0E94962EAA81BB810E9498
:105A8000622D11F00C941E2DC29A83E0481A8827CB
:105A9000580A24960895481A8827580A0895480EE7
:105AA0008827581E08950D911D912D913C9181E0FC
:105AB000080F8827181F281F381F3C932E931E930A
:105AC0000E930895ED91FC913196FC93EE93089519
:105AD000ED91FC913197FC93EE9308950D911D91FA
:105AE0002D913C9101501040204030403C932E932A
:105AF0001E930E9308954091DD025091DE020DE851
:105B000015E30E948F2D49E156E3040F151F009302
:105B1000DD021093DE02498158810C94B42D08D027
:105B20003DD000FC10D0089503D01ED001F8F9CF6D
:105B30000024E89457FF02C009D0689400F80BD005
:105B400010F80124089502D009D008955095409589
:105B50004F5F5F4F0895E89417FF089500951095E3
:105B60000F5F1F4F68940895352F242FE894452B1D
:105B700011F468940895512F402F0027112780E1D8
:105B8000440F551F001F111F021B130B416018F417
:105B9000020F131F4E7F8A9599F708950F92049F65
:105BA000202C312C419F300C509F030C022D102DC6
:105BB0000F900895C8950D9231960020D9F7089559
:105BC0008F938D918823E9F711978F91089581E044
:105BD0005F9B8827089588275F9B089500C05F9B7F
:105BE000FECF8CB10895A8E6B7E08D91882311F01F
:105BF00011D0FBCF08950E94C92E802D11F00AD03C
:105C0000FACF08958D9106D03A95E1F708958DE089
:105C100001D08AE05D9BFECF8CB9089588EE93E0B9
:105C2000A3D03197D9F7089550D00AD000FC05D001
:105C300008954BD020D001F8F9CF52D05AD0089512
:105C4000842F952FA62FB72F442755276627772710
:105C5000F1E2889409C020F4480F591F6A1F7B1F86
:105C60007695679557954795379527951795079595
:105C7000FA9589F70895842F952FA62FB72FE894CA
:105C8000452B462B472B11F468940895402F512F34
:105C9000622F732F0027112722273327F0E2440FAA
:105CA000551F661F771F001F111F221F331F081B60
:105CB000190B2A0B3B0B416028F4080F191F2A1FF0
:105CC0003B1F4E7FFA9559F708950024E89477FF1B
:105CD00002C006D0689400F809D010F80124089595
:105CE00012D04F5F5F4F6F4F7F4F0895E89437FF9B
:105CF000089500951095209530950F5F1F4F2F4FF9
:105D00003F4F68940895409550956095709508951B
:105D10003197F1F708950E94A72E8C910E94A92E29
:105D20008D939A95D1F70E94A82E08950E94A72ED0
:105D30008D910E94A92E9A95D9F70E94A82E0895B8
:105D4000BF9ABE98C69ABD9A80E58DB90895089508
:105D500008958FB9779BFECF8FB10895689462F84C
:105D60000895E89462F80895EF93FF93EE27E82BE7
:105D7000E92B31F0E0EDF7E03197F1F70197D1F73A
:105D8000FF91EF9108955A924A92480E8827581E23
:105D90000895C895319600200895819104D08D937F
:105DA0008823D9F70895813618F08B3708F48F7D52
:105DB000089580E30EF4839508952E2E3F2E9927A3
:105DC00081918D3209F093958823D1F79A95E22D30
:105DD000F32D112361F0091718F011F0101B01C009
:105DE000191B28F021F080E28D931A95E9F7808144
:105DF0008D3219F48D93319604C0222311F08BE279
:105E00008D93091738F031F0091B21F080E38D9351
:105E10000A95E9F781918D938823E1F7332351F0B7
:105E2000EA2FFB2F319633958E9182933A95E1F7C5
:105E30008EE28C930895040F151F261F371F0895B7
:105E4000041B150B260B370B08950417150726079F
:105E500037070895000F111F221F331F0895009563
:105E60001095209530950F5F1F4F2F4F3F4F08958E
:105E7000019110810EC001911191219130810BC0CF
:105E80000191108117FF05C03FEF2FEF04C0008183
:105E900011272227332737FF03C0E1DF8DE28D93DF
:105EA000CF93DF93CF92DF92EF92AA24BB24CC242E
:105EB000DD24EE2440E2CAE0DD2755E093E388814B
:105EC000890F87FD9F7083FD907F891B89935A9569
:105ED000A9F7C0DFAA1CBB1CCC1CDD1CEE1C4A951C
:105EE00051F7E894EFE0FF2782910ED0EB30E0F716
:105EF0001EF068948A2D0CD088278D93EF90DF9048
:105F0000CF90DF91CF910895982F829501D0892F5E
:105F10008F70805D26F0803309F4089568948D9326
:105F2000089588278D93089581918D938823E1F7B3
:105F3000089509919191992351F08A95D9F7319754
:105F400081918D930A9519F08823D1F70895E9CFAF
:105F5000E199FECFEEBBFFBB3196089591E001C001
:105F600092E07B3751F47FB7F894F2DF8D918DBBCF
:105F7000E29AE19A9A95C9F77FBF7727089591E051
:105F800001C092E0E5DFE09A8DB38D939A95D1F749
:105F90000895FF93881BF9E0001FFA9511F4FF9113
:105FA0000895881F841B18F4840F8894F5CF0894F3
:105FB000F3CF689401C0E894AF93BF938D9116F02E
:105FC000919103C00E94C92E902D891718F011F4E9
:105FD0008823A1F7BF91AF9108954D503353544199
:105FE0004D50205265616C6974792D53797320345A
:105FF0002E375049520053005000454570726F6D66
:1060000020002C004D4D4320696E6974200072659C
:10601000747279202E2E2E0044535020696E6974BC
:1060200020004F005A0059004B0055004700520015
:1060300057004100480021004E0042005800440033
:10604000450056004D00540049004C00434F4E4659
:10605000494700002000442000002E006F6B000024
:106060004E6F2063617264004261642063617264F8
:106070000000506172746974696F6E207479706584
:10608000203A0000506172746974696F6E207374F5
:106090006172743A0000536563742F636C75737496
:1060A000657220203A00526F6F74203A00005265EA
:1060B0006164206572726F72203100005265616404
:1060C000206572726F722032206F6E207365637468
:1060D0006F723A20000052656164206572726F72BF
:1060E0002033000052656164206572726F72203443
:1060F000000052656164206572726F722035000085
:0E610000526561642074696D656F75740000EE
:00000001FF
